:100000002BC072C144C043C042C041C040C03FC0C9
:100010003EC03DC03CC03BC03AC039C038C037C00C
:1000200036C0040309040E03460061006200490063
:100030005300500012011001FF00000881179F0CAF
:1000400004010002000109021200010100801409EC
:1000500004000000FF00000011241FBECFE5D1E026
:10006000DEBFCDBF10E0A0E6B0E0E2E4F8E002C001
:1000700005900D92A236B107D9F710E0A2E6B0E0E4
:1000800001C01D92A53AB107E1F7BFD3D8C3B8CFDD
:1000900085B7826085BF8BB780648BBF08951F933F
:1000A000CF93DF9360918B00635067FD9AC080917E
:1000B0008800CCE0D0E0C81BD109C157DF4F809148
:1000C00087008D3209F07BC0683009F088C083EC6E
:1000D00080937B008AE580936000109262008881A3
:1000E000807639F0CE017FD2282F8F3F09F456C099
:1000F0005CC09A81109284008981882321F4109237
:10010000850022E044C0853019F490938C003EC0F5
:10011000863069F58B81813019F484E390E004C066
:10012000823041F486E490E090938A0080938900C5
:1001300022E119C08330B1F4992341F482E290E0C6
:1001400090938A008093890024E00DC0913051F093
:10015000923041F486E290E090938A008093890087
:100160002EE001C020E080E4809362001EC0883051
:1001700021F421E08EE890E00CC0893019F49093CE
:100180008E0004C08A3011F421E001C020E084E830
:1001900090E090938A008093890007C0888187FD52
:1001A0002E8180E88093620006C08F81882319F435
:1001B0008E81821708F0822F8093610010C0809199
:1001C000620087FF0CC0CE01C7D28F3F21F48EE1C1
:1001D0008093600004C0882311F010926100109297
:1001E0008B008091600084FF58C0809161008F3F38
:1001F00009F453C0182F893008F018E0811B809350
:10020000610080917B0098E8892780937B0011230F
:1002100091F18091620087FF08C08CE790E0612F28
:1002200086D2182F893098F526C020918900309108
:100230008A0086FF0DC0ACE7B0E080E090E0F901F5
:10024000E80FF91FE491ED9301961817C1F708C064
:10025000912FD901ECE7F0E08D9181939150E1F776
:100260001150812F90E01F5F0196820F931F909392
:100270008A00809389008CE790E0612F31D0612F54
:100280006C5F6C3041F08FEF8093610004C08FEFA2
:10029000809361006EE16093600094E189B381789E
:1002A00031F49150D9F710928C0010928600DF91B2
:1002B000CF911F910895A82FB92F80E090E041E0E1
:1002C00050EA609530E009C02D9182279795879577
:1002D00010F084279527305EC8F36F5FA8F3089568
:1002E000EADF8D939D930895CF93CFB7CF93C395B6
:1002F000C89BE9F7C89B09C0C89B07C0C89B05C03D
:10030000C89B03C0C89B01C0A1C0DF93C0918800F7
:10031000DD27C157DF4FC89B02C0DF91EBCF2F9382
:100320000F931F9309B32FEF00FB20F94F933F93D7
:1003300019B34FEF012700FB21F93BE031C04E7F9D
:10034000012F19B3216028C0102F4D7F22600000BB
:1003500009B329C04B7F2460012F000019B32BC0C3
:1003600019B3477F28602AC04F7E09B320612CC093
:100370004F7D19B320622FC04F7B09B3206432C078
:10038000422709B349934FEF0000102710FB20F9D3
:1003900019B31178C9F1297F91F2012700FB21F9E6
:1003A00009B3237F89F2315058F1102710FB22F94D
:1003B00019B3277E79F2012700FB23F92F7C81F204
:1003C00009B3102710FB24F92F7971F200C019B37B
:1003D000012700FB25F92F7359F200C009B310273C
:1003E00010FB26F9223040F200C019B3012700FBB0
:1003F00027F9243028F64F77206819B30000F9CF89
:1004000010E41ABF002717C03B503195C31BD040E2
:1004100010E41ABF0881033CE9F00B34D9F02091B5
:1004200086001981110F1213EDCF093641F10D32FB
:1004300011F0013E39F700938D003F914F911F91CC
:100440000F912F91DF91CAB7C6FD51CFCF91CFBF8A
:10045000CF91189520918D00222379F310918B0074
:10046000112311F5343012F130938B002093870063
:10047000109188003BE0311B3093880017C0009139
:100480008B0001308CF40AE53091600034FD10C01F
:1004900000936000CBE7D0E00FC02795A8F451503F
:1004A000A9F4220F0000F9CF4AE503C042ED01C0D4
:1004B000432FC4E1D0E032E01AB31168D89A1ABBD6
:1004C0000BB320E411E85F93012756E00BBB27959F
:1004D00020F4515021F4220FF9CF012756E00000FB
:1004E0003B5A0BBBD0F2279528F4515029F4220F28
:1004F0000000F9CF012756E027950BBB20F451509F
:1005000021F4220FF9CF012756E0299133230BBBA9
:1005100021F60E7710918C00110FC651D0400BBB05
:1005200011F01093860010E41ABF01601AB31E7711
:10053000402F4E775F9100C000C00BBB1ABB4BBB76
:100540007CCFDC01FB016091630050E07D9190E085
:1005500040E820E030E0842F872309F0DE9A062E61
:1005600000C000000A94E1F7DC9A062E00C00000EB
:100570000A94E1F7990FCD999F5FDE98DC98469534
:100580002F5F3F4F2830310531F790835F5F543044
:1005900011F03196DBCF089520916600309167000D
:1005A0002F5F3F4F3093670020936600215030400B
:1005B00080916A0087FF02C0220F331F80936B0077
:1005C00020FF03C0886080936B00832F8695809303
:1005D0006C003695279520936D008BE690E06FE6D2
:1005E00070E0AFDF08950F931F93CF93DF93EC017B
:1005F00039813323B9F420E030E0F901ED58FF4FA1
:10060000DE01A20FB31F8C9180832F5F3F4F2830F4
:10061000310599F783E790E090938A0080938900F1
:1006200088E080C05C81E52FF0E0313059F48081B2
:100630008093730083E790E090938A008093890011
:1006400081E070C0323011F48A8112C0BC016E5F4B
:100650007F4F4A81242F277081E090E0982F01C0BE
:10066000990F2A95EAF7333029F4909580818923F0
:10067000808357C0343019F48081892BF9CF35300D
:1006800079F440936300552311F09AE001C092E0A1
:100690008AB38A658ABB8BB3857A982B9BBB41C092
:1006A000363041F4DB9A8BB3857A8BBB8AB3857A7B
:1006B0008ABB37C08BB38823A1F1373059F403E7E5
:1006C00010E0CB01B8013DDF10938A000093890050
:1006D00084E028C0383031F4409364008B818093EB
:1006E00065001FC08C819D81909367008093660098
:1006F000393011F480E211C03B3011F480EA0DC0B2
:100700008A819B8190936900809368003A3011F44C
:1007100080E403C03C3029F480EC80936A008FEFC2
:1007200001C080E0DF91CF911F910F9108950F9349
:100730001F93CF93DF93062FEC0110E005C02CDF51
:100740008091720089931F5F1017C8F3802FDF918B
:10075000CF911F910F9108957F928F929F92AF92A8
:10076000BF92CF92DF92EF92FF920F931F93CF939E
:10077000DF93862EA0906800B0906900909064008E
:10078000C090650020916300E22EFF2435E0EE0C5E
:10079000FF1C3A95E1F78C01DD2420E6722E24C07F
:1007A000F801808180936E00F7DE80916B008725D1
:1007B00080936B00C0E0D0E011C08BE690E06FE664
:1007C00070E0BFDE9091720080916E00981721F466
:1007D000991511F09C1529F4CE0DDF1DCA15DB0506
:1007E00060F3D3940F5F1F4FD814D0F281E0DF91F4
:1007F000CF911F910F91FF90EF90DF90CF90BF901E
:10080000AF909F908F907F9008952EE088E190E0C8
:100810000FB6F894A89581BD0FBE21BD39DCD09AE2
:1008200020E048EB5BE004C0A895CA010197F1F70E
:100830002150D1F7D0987894A89531DCFDCFF89469
:02084000FFCFE8
:020842005AFF5B
:00000001FF
